:020000040000FA
:1000000048EF21F0C96E12007EEF1DF0E0EC0FF01A
:100010000DEC1BF0FDD71200BEEF1FF0D9CFE5FFAE
:10002000E1CFD9FF00C0E5FF01C0E5FF02C0E5FF59
:1000300003C0E5FF04C0E5FF05C0E5FF06C0E5FF1E
:1000400007C0E5FF08C0E5FF09C0E5FF0AC0E5FFFE
:100050000BC0E5FF0CC0E5FF0DC0E5FF0EC0E5FFDE
:100060000FC0E5FF10C0E5FF11C0E5FF12C0E5FFBE
:1000700013C0E5FF14C0E5FF15C0E5FF16C0E5FF9E
:1000800017C0E5FF18C0E5FF19C0E5FF1AC0E5FF7E
:100090001BC0E5FF1CC0E5FF1DC0E5FF1EC0E5FF5E
:1000A000020EDBCF00F0030EDBCF01F0040EDBCF3E
:1000B00002F0050EDBCF03F0060EDBCF04F0070ED7
:1000C000DBCF05F0080EDBCF06F0090EDBCF07F023
:1000D0000A0EDBCF08F0096A0A6A02C00DF00D5063
:1000E000800A0DE102500F012B6F01502A6F005062
:1000F000296F0F0E016E290E006E800E026E03C076
:10010000E9FF04C0F3FF055081EC21F00B6E0B50AA
:10011000D8B4FCEF03F00B50250A02E0E3EF03F044
:100120000C6A0D6A0E6A0F6A106A0A0E116E126A64
:10013000136A146A200E156E1668176A2B0E186E55
:10014000032A02E3044A052A03C0E9FF04C0F3FFBF
:10015000055081EC21F0196E250A13E11950E56E66
:100160000250E56E0150E56E0050E56E85EC15F02D
:10017000040EE126094A0A2A032A02E3044A052A50
:10018000BED71950300A06E1300E156E032A02E37D
:10019000044A052A03C0E9FF04C0F3FF055081ECBF
:1001A00021F02D0A06E1010E146E032A02E3044A2F
:1001B000052A03C0E9FF04C0F3FF055081EC21F0DC
:1001C000200A08E1010E176E200E186E032A02E3C2
:1001D000044A052A03C0E9FF04C0F3FF055081EC7F
:1001E00021F02B0A06E1010E176E032A02E3044AEE
:1001F000052A03C0E9FF04C0F3FF055081EC21F09C
:10020000196E800F4F0F2DE31950800F460F29E212
:1002100003C019F004C01AF005C01BF019C0E9FFB3
:100220001AC0F3FF1B5081EC21F01C6E800F500FA1
:1002300012E31C50800F460F0EE213500A0DF3CF4D
:100240001DF01D501C26D00E1C24136E192A02E32B
:100250001A4A1B2AE3D719C003F01AC004F01BC0C6
:1002600005F003C0E9FF04C0F3FF055081EC21F065
:100270002E0A2EE1032A02E3044A052A166A03C065
:1002800019F004C01AF005C01BF019C0E9FF1AC02C
:10029000F3FF1B5081EC21F01C6E800F500F12E316
:1002A0001C50800F460F0EE216500A0DF3CF1DF0C2
:1002B0001D501C26D00E1C24166E192A02E31A4A61
:1002C0001B2AE3D719C003F01AC004F01BC005F0C5
:1002D00003C0E9FF04C0F3FF055081EC21F0196E63
:1002E0006C0A07E1010E0C6E032A02E3044A052A98
:1002F00009D01950680A06E1010E0E6E032A02E3C6
:10030000044A052A03C0E9FF04C0F3FF055081EC4D
:1003100021F0750A06E1010E106E032A02E3044A79
:10032000052A03C0E9FF04C0F3FF055081EC21F06A
:10033000196E730A05E1010E0D6E200E156E3FD089
:100340001950780A03E1100E116E39D01950580A6D
:1003500005E1100E116E010E126E31D01950630AB4
:1003600002E1116A2CD019506F0A03E1080E116ED8
:1003700026D01950660A03E1010E0F6E20D01950E5
:10038000640A1DE01950690A1AE0105005E0FF0EDA
:1003900003260422052213D01950E56E0250E56EA3
:1003A0000150E56E0050E56E85EC15F0040EE12677
:1003B000094A0A2A032A02E3044A052AA0D60D5054
:1003C00021E00650030F0D6E000E0720196E000E7F
:1003D00008201A6E0DC006F019C007F01AC008F008
:1003E000FD0E0D26FF0E19221A220DC0E9FF19C0BD
:1003F000F3FF1A505DEC20F00D6EF3CF19F0F4CF3F
:100400001AF032D10F50D8B43ED00650040F0F6E00
:10041000000E07201B6E000E08201C6E0FC006F099
:100420001BC007F01CC008F0FC0E0F26FF0E1B229D
:100430001C220FC0E9FF1BC0F3FF1C50E3EC1FF0B0
:100440000F6EF3CF1BF0F4CF1CF0E9CF1DF0040EBC
:10045000196E000E0D6E800E1A6E1650E56E240E8B
:10046000E56E040EE56E000EE56E1D50E56E1C5047
:10047000E56E1B50E56E0F50E56EC4EC0DF0080EF6
:10048000E1261668F1D016680C5023E00650040FE0
:100490000C6E000E07200F6E000E08201B6E0CC0A5
:1004A00006F00FC007F01BC008F0FC0E0C26FF0E74
:1004B0000F221B220CC0E9FF0FC0F3FF1B50E3EC1F
:1004C0001FF00C6EF3CF0FF0F4CF1BF0E9CF1CF050
:1004D0006AD00E5032E00650020F0E6E000E07205A
:1004E0001D6E000E08201E6E0EC006F01DC007F027
:1004F0001EC008F0FE0E0E26FF0E1D221E220EC08C
:10050000E9FF1DC0F3FF1E501CEC21F00E6E0EC063
:100510000CF0E86A0EBEFF0E0F6E1B6E1C6E1150C3
:100520000A0A03E11050D8B43ED00C500E6E0EC033
:100530000CF00F6A1B6A1C6A36D00650020F0E6E52
:10054000000E07201D6E000E08201E6E0EC006F065
:100550001DC007F01EC008F0FE0E0E26FF0E1D2265
:100560001E220EC0E9FF1DC0F3FF1E501CEC21F03F
:100570000E6EF3CF1DF00EC00CF01DC00FF0E86A38
:100580001DBEFF0E1B6E1C6E11500A0A02E11050B8
:100590000AE00C500E6E0F501D6E0EC00CF01DC008
:1005A0000FF01B6A1C6A040E196E010E0D6E800E90
:1005B0001A6E1150D8B440D0105013E01150E56EAF
:1005C000040EE56E010EE56E1C50E56E1B50E56EE7
:1005D0000F50E56E0C50E56EEAEC11F0070EE126C7
:1005E00012D01150E56E040EE56E010EE56E1C5042
:1005F000E56E1B50E56E0F50E56E0C50E56EBBECE2
:1006000018F0070EE12617502FE00DC0E9FF19C0C2
:10061000F3FF1A5081EC21F02D0A26E0FF0E0D2683
:1006200019221A2218C0E5FF0DC0E9FF19C0F3FF17
:100630001A500EEC22F018D00CC0E5FF0DC0E9FFF7
:1006400019C0F3FF1A500EEC22F00D50010F0C6E82
:10065000000E19200E6E000E1A20E56A0CC0E9FF8C
:100660000EC0F3FF0EEC22F00DC00CF019C00EF01E
:100670001AC00FF013C010F0105010E00CC0E9FFCA
:100680000EC0F3FF0F5081EC21F0176E175006E0FB
:100690000C2A02E30E4A0F2A1006EED710C013F000
:1006A00014501EE109C00CF00AC00EF010C00FF08B
:1006B0000F5010E01550E56E0250E56E0150E56EEA
:1006C0000050E56E85EC15F0040EE1260C4A0E2A6A
:1006D0000F06EED70CC009F00EC00AF00FC013F0E1
:1006E00016C00CF00DC00DF019C00EF01AC00FF0BE
:1006F00009C010F00AC015F00DC0E9FF0EC0F3FFED
:100700000F5081EC21F0166E1650D8B43ED00CC0BC
:1007100016F0176A161E171E1650171005E00CC0AB
:1007200016F00C06165031E00DC0E9FF0EC0F3FFC5
:100730000F5081EC21F0116E125010E01150E56E57
:10074000D9EC20F0166EE652165004E01150166EE9
:10075000169A02D011C016F016C011F01150E56EB5
:100760000250E56E0150E56E0050E56E85EC15F027
:10077000040EE1260D2A02E30E4A0F2A104A152A1A
:100780001350D8B4B9D71306B7D710C009F015C0A5
:100790000AF014502BE010C00CF015C00DF013C07F
:1007A0000EF00E501FE0200EE56E0250E56E015077
:1007B000E56E0050E56E85EC15F0040EE1260C4A5E
:1007C0000D2A0E06EED70B50E56E0250E56E015075
:1007D000E56E0050E56E85EC15F0040EE126094A41
:1007E0000A2A04D00CC009F00DC00AF0032A02E363
:1007F000044A052A7FEF00F00AC0F3FF0950E4CF56
:100800001EF0E4CF1DF0E4CF1CF0E4CF1BF0E4CFEA
:100810001AF0E4CF19F0E4CF18F0E4CF17F0E4CFEA
:1008200016F0E4CF15F0E4CF14F0E4CF13F0E4CFEA
:1008300012F0E4CF11F0E4CF10F0E4CF0FF0E4CFEA
:100840000EF0E4CF0DF0E4CF0CF0E4CF0BF0E4CFEA
:100850000AF0E4CF09F0E4CF08F0E4CF07F0E4CFEA
:1008600006F0E4CF05F0E4CF04F0E4CF03F0E4CFEA
:1008700002F0E4CF01F0E4CF00F0E4CFD9FF1200A2
:1008800005C0E5FF06C0E5FF07C0E5FF08C0E5FFBE
:1008900009C0E5FF0AC0E5FF0BC0E5FF0CC0E5FF9E
:1008A0000DC0E5FF0EC0E5FF0FC0E5FF10C0E5FF7E
:1008B00011C0E5FF12C0E5FF13C0E5FF14C0E5FF5E
:1008C00015C0E5FF16C0E5FF17C0E5FF18C0E5FF3E
:1008D00019C0E5FF1AC0E5FF1BC0E5FF1CC0E5FF1E
:1008E0001DC0E5FF000E00B0050F066AF60F02E31B
:1008F000062AFCD70A0F056E042E03D0FB0F01E376
:10090000062A065000B0020F00B2050F076AF60F64
:1009100002E3072AFCD70A0F066E042E03D0FB0F52
:1009200001E3072A075000B0060F00B2020F00B41F
:10093000050F086AF60F02E3082AFCD70A0F076EB4
:10094000042E03D0FB0F01E3082A085000B2010F68
:1009500000B4020F00B6050F096AF60F02E3092A78
:10096000FCD70A0F086E042E03D0FB0F01E3092AFF
:10097000095000B0090F00B2080F00B4060F00B60E
:10098000020F00B8050F0A6AF60F02E30A2AFCD725
:100990000A0F096E042E03D0FB0F01E30A2A0A5046
:1009A00000B0030F00B2070F00B4050F00B6010F2F
:1009B00000B8020F00BA050F0B6AF60F02E30B2A0C
:1009C000FCD70A0F0A6E042E03D0FB0F01E30B2A9B
:1009D0000B5000B0050F00B4010F00B6030F00B8B4
:1009E000060F00BA020F00BC050F0C6AF60F02E3F7
:1009F0000C2AFCD70A0F0B6E042E03D0FB0F01E369
:100A00000C2A0C5000B0070F00B2050F00BA010FFE
:100A100000BC020F00BE050F0D6AF60F02E30D2A9F
:100A2000FCD70A0F0C6E042E03D0FB0F01E30D2A36
:100A30000D5000B0070F00B2050F00B4010F00B653
:100A4000020F00B8040F00BA080F00BC060F00BE6A
:100A5000020F01B0050F0E6AF60F02E30E2AFCD753
:100A60000A0F0D6E042E03D0FB0F01E30E2A0E5069
:100A700000B0040F00B2090F00B4090F00B6080F50
:100A800000B8060F00BA020F00BC050F00BE010F30
:100A900001B0020F01B2050F0F6AF60F02E30F2A31
:100AA000FCD70A0F0E6E042E03D0FB0F01E30F2AB2
:100AB0000F5000B0040F00B2080F00B4070F00B6CB
:100AC000050F00B8010F00BA030F00BC060F00BEEF
:100AD000030F01B0060F01B2020F01B4050F106A37
:100AE000F60F02E3102AFCD70A0F0F6E042E03D074
:100AF000FB0F01E3102A105000B0060F00B2020FE6
:100B000000B4050F00B6010F00B8030F00BA060FBE
:100B100000BC020F00BE050F01B2010F01B4020FAD
:100B200001B6050F116AF60F02E3112AFCD70A0F6E
:100B3000106E042E03D0FB0F01E3112A115000B0F8
:100B4000040F00B2090F00B4080F00B6070F00B879
:100B5000040F00BA080F00BC070F00BE040F01B05D
:100B6000090F01B2080F01B4060F01B6020F01B858
:100B7000050F126AF60F02E3122AFCD70A0F116E54
:100B8000042E03D0FB0F01E3122A125000B4010F10
:100B900000B6030F00B8070F00BA040F00BC090F1E
:100BA00000BE090F01B0080F01B2070F01B4050F15
:100BB00001B6010F01B8020F01BA050F136AF60F53
:100BC00002E3132AFCD70A0F126E042E03D0FB0F88
:100BD00001E3132A135000B0060F00B2020F00B455
:100BE000040F00B6080F00B8060F00BA030F00BCD0
:100BF000060F00BE030F01B0070F01B2050F01B4CD
:100C0000010F01B6030F01B8060F01BA020F01BCB4
:100C1000050F146AF60F02E3142AFCD70A0F136EAD
:100C2000042E03D0FB0F01E3142A145000B0090F67
:100C300000B2090F00B4080F00B6060F00B8030F8A
:100C400000BA070F00BC040F00BE090F01B0080F67
:100C500001B2070F01B4050F01BA010F01BC020F69
:100C600001BE050F156AF60F02E3152AFCD70A0F1D
:100C7000146E042E03D0FB0F01E3152A155000B0AB
:100C8000050F00B2010F00B4030F00B6070F00B844
:100C9000050F00BC010F00BE020F01B0050F01B22D
:100CA000010F01B4030F01B6070F01B8040F01BA19
:100CB000080F01BC060F01BE020F02B0050F166A35
:100CC000F60F02E3162AFCD70A0F156E042E03D086
:100CD000FB0F01E3162A165000B2010F00B4020FF9
:100CE00000B6040F00B8090F00BA090F00BC080FC6
:100CF00000BE060F01B0020F01B2050F01B8010FCF
:100D000001BA020F01BC050F01BE010F02B0020FB4
:100D100002B2050F176AF60F02E3172AFCD70A0F73
:100D2000166E042E03D0FB0F01E3172A175000BAEA
:100D3000010F00BC030F00BE070F01B0050F01B487
:100D4000010F01B6020F01B8040F01BA080F01BC70
:100D5000060F01BE030F02B0060F02B2020F02B46B
:100D6000050F186AF60F02E3182AFCD70A0F176E50
:100D7000042E03D0FB0F01E3182A185001B0010F15
:100D800001B2030F01B4060F01B6020F01B8040F40
:100D900001BA080F01BC070F01BE050F02B2010F17
:100DA00002B4020F02B6050F196AF60F02E3192A00
:100DB000FCD70A0F186E042E03D0FB0F01E3192A8B
:100DC000195001B6010F01B8020F01BA040F01BC9E
:100DD000090F01BE090F02B0090F02B2080F02B4D9
:100DE000060F02B6020F02B8050F1A6AF60F02E3E9
:100DF0001A2AFCD70A0F196E042E03D0FB0F01E349
:100E00001A2A1A5001BE010F02B0030F02B2070FD7
:100E100002B4050F02B6010F02B8020F02BA050FA5
:100E20001B6AF60F02E31B2AFCD70A0F1A6E042E68
:100E300003D0FB0F01E31B2A1B5002B4010F02B6C3
:100E4000030F02B8060F02BA020F02BC050F1C6A9C
:100E5000F60F02E31C2AFCD70A0F1B6E042E03D0E8
:100E6000FB0F01E31C2A1C5002BA010F02BC020F47
:100E700002BE050F1D6AF60F02E31D2AFCD70A0FFA
:100E80001C6E042E03D0FB0F01E31D2A300FEE6E03
:100E90001B50300FEE6E1A50300FEE6E1950300F9F
:100EA000EE6E1850300FEE6E1750300FEE6E16507B
:100EB000300FEE6E1550300FEE6E1450300FEE6E98
:100EC0001350300FEE6E1250300FEE6E1150300F87
:100ED000EE6E1050300FEE6E0F50300FEE6E0E5063
:100EE000300FEE6E0D50300FEE6E0C50300FEE6E78
:100EF0000B50300FEE6E0A50300FEE6E0950300F6F
:100F0000EE6E0850300FEE6E0750300FEE6E06504A
:100F1000300FEE6E0550300FEE6E170EE4CF1DF061
:100F2000E4CF1CF0E4CF1BF0E4CF1AF0E4CF19F0CB
:100F3000E4CF18F0E4CF17F0E4CF16F0E4CF15F0CB
:100F4000E4CF14F0E4CF13F0E4CF12F0E4CF11F0CB
:100F5000E4CF10F0E4CF0FF0E4CF0EF0E4CF0DF0CB
:100F6000E4CF0CF0E4CF0BF0E4CF0AF0E4CF09F0CB
:100F7000E4CF08F0E4CF07F0E4CF06F0E4CF05F0CB
:100F8000120000C0E5FF01C0E5FF02C0E5FF03C09D
:100F9000E5FF04C0E5FF05C0E5FF06C0E5FF07C0AB
:100FA000E5FF08C0E5FF09C0E5FF0AC0E5FF0BC08B
:100FB000E5FF006A016A040E015CD8B0E8D10A01BD
:100FC0004E2B100E4E5D01E34E6B0A014E39E84484
:100FD0001F0B026E036A2E0E02260F0E032202C0A2
:100FE000E9FF03C0EAFFEFCF02F0070E4E15036ED4
:100FF000010E046E000E056E035006E0E86CD890FA
:1010000004360536010FFCE3066A0250041606504A
:101010000516045005E1055003E1046A042A01D0D5
:10102000046A0450D880E866D890046A04360450F4
:10103000D8B4C1D70A014E51020DF450036EF3CF5C
:1010400002F0E00E0224046E000E0320056E04C0C0
:10105000E9FF05C0EAFFEECF04F0EFCF05F00A018B
:101060004BA19DD0B30E0224066E040E0320076E22
:1010700006C0E9FF07C0EAFFEECF06F0EFCF07F0AA
:101080000550800FF36E0750800FF35C02E10650AD
:10109000045C03E2046A056A60D0D30E0226040EE3
:1010A000032202C0E9FF03C0EAFFEECF02F0EFCF58
:1010B00003F00350800FF36E0550800FF35C02E1E4
:1010C0000450025C04E204683F0E056E46D00650F0
:1010D000045C086E07500558096EE86A09BEFF0EE9
:1010E0000A6EE56E0A50E56E0950E56E0850E56E31
:1010F000E56AE56A400EE56E000EE56AD6EC0EF094
:10110000086EF3CF09F0F4CF0AF0E9CF0BF0080E28
:10111000E1260650025C066E07500358076EE86A27
:1011200007BEFF0E026EE56E0250E56E0750E56EDB
:101130000650E56E0B50E56E0A50E56E0950E56EFF
:101140000850E56EE6EC13F0026EF3CF03F0080EE4
:10115000E1260250046E0350056E0A014A51800FC9
:10116000F36E0550800FF35C02E10450495D03E328
:10117000046A056A14D00A014951FF08026E3F0E45
:101180004A55036E0550800FF36E0350800FF35CD9
:1011900002E10250045C03E304683F0E056E0A019D
:1011A0004E51020DF450036EF3CF02F0930E02265F
:1011B000040E032202C0E9FF03C0EAFFEECF02F0F3
:1011C000EFCF03F00250045C026E03500558036E2B
:1011D000D88003AED89004E3031E026CD8B4032A6F
:1011E000012A0A014A51800FF36E0350800FF35C0D
:1011F00002E10250495DD8B0DED60A014E51020D1F
:10120000F450076EF3CF06F0930E0626040E072265
:1012100006C0E9FF07C0EAFF04C0EEFF05C0EFFF0C
:101220000A014BA55AD00A014E51020DF450076E27
:10123000F3CF06F0000E0624086E0A0E0720096E92
:1012400008C0E9FF09C0EAFFEECF0AF0EFCF0BF0CC
:101250000A500B10D8B441D05C0E0626040E0722AB
:1012600006C0E9FF07C0EAFFEECF06F0EFCF07F0B8
:101270000650045C026E07500558036E02101CE015
:101280000350800F800F02E1010E025C066A0636F1
:101290000B50800F800F02E1010E0A5C0A6A0A36C9
:1012A00006500A1809E108C0E9FF09C0EAFF02C0B8
:1012B000EEFF03C0EFFF7FD60A014E51020DF4503E
:1012C000036EF3CF02F0000E02260A0E032202C0C4
:1012D000E9FF03C0EAFFEE6AEF6A0A014BA343D0BD
:1012E00000500EE100C002F0002A036A4F0E0226F1
:1012F0000A0E032202C0E9FF03C0EAFF420EEF6EAE
:1013000000C002F0002A036A4F0E02260A0E0322D2
:10131000640E0A014E25066E02C0E9FF03C0EAFF13
:1013200006C0EFFF00C002F0002A036A4F0E02263B
:101330000A0E03220550066E02C0E9FF03C0EAFF51
:1013400006C0EFFF00C002F0002A036A4F0E02261B
:101350000A0E03220450066E02C0E9FF03C0EAFF32
:1013600006C0EFFF28D64ECA02F00550E56E0450C5
:10137000E56EE56A0250E56E000EE56E2D0EE56E37
:10138000FA0EE56ED9EC1BF0070EE12614D60050DC
:101390001DE00A014BA31AD000C002F0002A036A24
:1013A0004F0E02260A0E032202C0E9FF03C0EAFF25
:1013B0000A0EEF6E0050E56E800EE56E0A0EE56EC9
:1013C0004F0EE56E0EEC16F0040EE1260150E4CF50
:1013D0000BF0E4CF0AF0E4CF09F0E4CF08F0E4CF5B
:1013E00007F0E4CF06F0E4CF05F0E4CF04F0E4CF5B
:1013F00003F0E4CF02F0E4CF01F0E4CF00F01200FC
:1014000000C0E5FF01C0E5FF02C0E5FF03C0E5FF46
:1014100004C0E5FF05C0E5FF06C0E5FF07C0E5FF26
:1014200008C0E5FF09C0E5FF0AC0E5FF0BC0E5FF06
:101430000CC0E5FF0DC0E5FF0EC0E5FF000E00B0DB
:10144000010F00B2020F00B4040F00B6080F00B87D
:10145000060F00BA020F00BC040F00BE080F01B057
:10146000060F01B2020F01B4040F01B6080F01B854
:10147000060F01BA020F01BC040F01BE080F02B033
:10148000060F02B2020F02B4040F02B6080F02B830
:10149000060F02BA020F02BC040F02BE080F056A53
:1014A000F60F02E3052AFCD70A0F046E055000B8B8
:1014B000010F00BA030F00BC060F00BE020F01B0FF
:1014C000050F01B2010F01B4020F01B6040F01B8FC
:1014D000090F01BA090F01BC080F01BE060F02B0C7
:1014E000030F02B2070F02B4040F02B6080F02B8CE
:1014F000070F02BA050F066AF60F02E3062AFCD7A9
:101500000A0F056E065000BE010F01B0020F01B2B6
:10151000050F01BA010F01BC030F01BE070F02B096
:10152000050F02B4010F02B6020F02B8050F02BA8E
:10153000010F02BC030F02BE060F076AF60F02E39B
:10154000072AFCD70A0F066E075001B4010F01B637
:10155000020F01B8040F01BA080F01BC060F01BE4B
:10156000020F02B0050F02B2010F02B4020F02B661
:10157000040F02B8080F02BA070F02BC040F02BE24
:10158000080F086AF60F02E3082AFCD70A0F076E55
:10159000085001BC010F01BE030F02B0060F02B2DA
:1015A000030F02B4060F02B6020F02B8040F02BA0C
:1015B000090F02BC090F02BE080F096AF60F02E309
:1015C000092AFCD70A0F086E095002B2010F02B4B3
:1015D000020F02B6050F02BC010F02BE030F0A6A1A
:1015E000F60F02E30A2AFCD70A0F096E0A5002B866
:1015F000010F02BA020F02BC040F02BE080F0B6AF1
:10160000F60F02E30B2AFCD70A0F0A6E0B500E6A84
:101610000EE10A5010E1095012E1085014E10750A0
:1016200016E1065018E105501AE104501CD00E2AAC
:10163000300FEE6E0A500E2A300FEE6E09500E2A51
:10164000300FEE6E08500E2A300FEE6E07500E2A45
:10165000300FEE6E06500E2A300FEE6E05500E2A39
:10166000300FEE6E04500E2A300FEE6E0E50E4CFA7
:101670000EF0E4CF0DF0E4CF0CF0E4CF0BF0E4CFAC
:101680000AF0E4CF09F0E4CF08F0E4CF07F0E4CFAC
:1016900006F0E4CF05F0E4CF04F0E4CF03F0E4CFAC
:1016A00002F0E4CF01F0E4CF00F01200800EE56E0E
:1016B000040EE56ED30EE56E26EC1AF0030EE1265D
:1016C000800EE56E040EE56EB30EE56E26EC1AF0A4
:1016D000030EE126800EE56E040EE56ED50EE56E76
:1016E00026EC1AF0030EE126800EE56E040EE56E80
:1016F000B50EE56E26EC1AF0030EE126800EE56EBF
:10170000040EE56ED70EE56E26EC1AF0030EE12608
:10171000800EE56E040EE56EB70EE56E26EC1AF04F
:10172000030EE126800EE56E040EE56ED90EE56E21
:1017300026EC1AF0030EE126800EE56E040EE56E2F
:10174000B90EE56E26EC1AF0030EE126800EE56E6A
:10175000040EE56EDB0EE56E26EC1AF0030EE126B4
:10176000800EE56E040EE56EBB0EE56E26EC1AF0FB
:10177000030EE126800EE56E040EE56EDD0EE56ECD
:1017800026EC1AF0030EE126800EE56E040EE56EDF
:10179000BD0EE56E26EC1AF0030EE126800EE56E16
:1017A000040EE56EDF0EE56E26EC1AF0030EE12660
:1017B000800EE56E040EE56EBF0EE56E26EC1AF0A7
:1017C000030EE126800EE56E040EE56EE10EE56E79
:1017D00026EC1AF0030EE126800EE56E040EE56E8F
:1017E000C10EE56E26EC1AF0030EE126800EE56EC2
:1017F000040EE56EE30EE56E26EC1AF0030EE1260C
:10180000800EE56E040EE56EC30EE56E26EC1AF052
:10181000030EE126800EE56E040EE56EE50EE56E24
:1018200026EC1AF0030EE126800EE56E040EE56E3E
:10183000C50EE56E26EC1AF0030EE126800EE56E6D
:10184000040EE56EE70EE56E26EC1AF0030EE126B7
:10185000800EE56E040EE56EC70EE56E26EC1AF0FE
:10186000030EE126800EE56E040EE56EE90EE56ED0
:1018700026EC1AF0030EE126800EE56E040EE56EEE
:10188000C90EE56E26EC1AF0030EE126800EE56E19
:10189000040EE56EEB0EE56E26EC1AF0030EE12663
:1018A000800EE56E040EE56ECB0EE56E26EC1AF0AA
:1018B000030EE126800EE56E040EE56EED0EE56E7C
:1018C00026EC1AF0030EE126800EE56E040EE56E9E
:1018D000CD0EE56E26EC1AF0030EE126800EE56EC5
:1018E000040EE56EEF0EE56E26EC1AF0030EE1260F
:1018F000800EE56E040EE56ECF0EE56E26EC1AF056
:10190000030EE126800EE56E040EE56EF10EE56E27
:1019100026EC1AF0030EE126800EE56E040EE56E4D
:10192000D10EE56E26EC1AF0030EE126120000C07F
:10193000E5FF01C0E5FF02C0E5FF03C0E5FF04C00D
:10194000E5FF05C0E5FF06C0E5FF07C0E5FF08C0ED
:10195000E5FF09C0E5FFC2B202D10A014D51D8B47A
:10196000ADD00A014C51020DF450016EF3CF00F0DE
:10197000E00E0026000E012200C0E9FF01C0EAFFD0
:10198000EECF02F0EFCF03F003340330056E0230E8
:10199000046E053405320432053405320432045035
:1019A000025C046E05500358056EC3CF06F0076A4B
:1019B0000650042607500522C4CF06F00650096ED3
:1019C000086A085004260950052200C0E9FF01C03A
:1019D000EAFF04C0EEFF05C0EFFF0A014851010A0B
:1019E00001E06AD00A014C51020DF450016EF3CFB0
:1019F00000F0E00E0024046E000E0120056E04C00D
:101A0000E9FF05C0EAFFEECF02F0EFCF03F0B30E1F
:101A10000026040E012200C0E9FF01C0EAFFEECF5C
:101A200004F0EFCF05F09C0E0426D8A00506035065
:101A3000800FF36E0550800FF35C02E10450025CEE
:101A40000EE20250640F046E000E0320056E00C00B
:101A5000E9FF01C0EAFF04C0EEFF05C0EFFF0A0185
:101A60004C51020DF450016EF3CF00F0D30E00265E
:101A7000040E012200C0E9FF01C0EAFFEECF04F02E
:101A8000EFCF05F0640E0426D8B0052A0550800F6C
:101A9000F36E0350800FF35C02E10250045C0CE231
:101AA0009C0E0226D8A0030600C0E9FF01C0EAFF91
:101AB00002C0EEFF03C0EFFF0A014D6B0A014C2B81
:101AC000100E4C5D01E34C6B0A014C39E8441F0BCE
:101AD000006E016A2E0E00260F0E012200C0E9FFE3
:101AE00001C0EAFFEFCF00F0070E4C15016E010EAA
:101AF000026E000E036E015006E0E86CD8900236CC
:101B00000336010FFCE3046A00500216045003166A
:101B1000025005E1035003E1026A022A01D0026A81
:101B20000250D880E866D890026A0236025017E068
:101B3000240E0A014C25006E016A040E012200C029
:101B4000E9FF01C0EAFFEFCF00F00044E844FC0BDE
:101B5000016E0128C26EC282010E0A014D6FE4CFF0
:101B600009F0E4CF08F0E4CF07F0E4CF06F0E4CFCB
:101B700005F0E4CF04F0E4CF03F0E4CF02F0E4CFCB
:101B800001F0E4CF00F01200D9CFE5FFE1CFD9FF9B
:101B900000C0E5FF01C0E5FF02C0E5FF03C0E5FFAF
:101BA00004C0E5FF05C0E5FF06C0E5FF07C0E5FF8F
:101BB00008C0E5FF09C0E5FF0AC0E5FF0BC0E5FF6F
:101BC000020EDBCF00F0030EDBCF01F0040EDBCF03
:101BD00002F0050EDBCF03F0060EDBCF04F0070E9C
:101BE000DBCF05F0080EDBCF06F0090EDBCF07F0E8
:101BF00006C008F0060608500EE006500424086EE1
:101C0000E86A06BEE8680520096E08C0E9FF09C059
:101C1000EAFFEF6AEDD700500401FB6F0150FC6F43
:101C20000250FD6F0350FE6FFBC400F0FCC401F0D6
:101C3000FDC402F0FEC403F0066A086A096A800E59
:101C400003140A6E065007E1085005E1095003E14C
:101C50000A50800A01E012D0039E00500401FB6F7D
:101C60000150FC6F0250FD6F0350FE6F04C0E9FF8E
:101C700005C0EAFF2D0EEF6E044A052A0401FD356A
:101C8000FE357E08006EFB51016EFC51026E7F0E28
:101C9000FD15036E066A038E086A096A0A6A0B6AF2
:101CA000005019E0D88000AED8900EE30850082606
:101CB00009360A360B3603BE08800150012602366B
:101CC00003360636002AECD7D890063203320232A9
:101CD00001320006E5D7085009100A100B1012E077
:101CE0000550E56E0450E56E0B50E56E0A50E56E4A
:101CF0000950E56E0850E56E7DEC1EF0006E060E94
:101D0000E12608D004C0E9FF05C0EAFF300EEF6EFF
:101D1000010E006E00500426E86A00BEE868052245
:101D2000075028E004C0E9FF05C0EAFF2E0EEF6E61
:101D3000002A044A052A07501808E56E0550E56E8A
:101D40000450E56E0650E56E0350E56E0250E56EF8
:101D50000150E56EEAEC1DF0016E070EE126015020
:101D6000002607500426E86A052204C0E9FF05C0E2
:101D7000EAFFEF6A0050E4CF0BF0E4CF0AF0E4CFC3
:101D800009F0E4CF08F0E4CF07F0E4CF06F0E4CFA9
:101D900005F0E4CF04F0E4CF03F0E4CF02F0E4CFA9
:101DA00001F0E4CF00F0E4CFD9FF1200D9CFE5FF76
:101DB000E1CFD9FF00C0E5FF01C0E5FF02C0E5FFAC
:101DC00003C0E5FF04C0E5FF05C0E5FF06C0E5FF71
:101DD00007C0E5FF020EDBCF00F0030EDBCF01F002
:101DE000040EDBCF02F0050EDBCF03F0060EDBCFD7
:101DF00004F0070EDBCF05F0080EDBCF06F0090E6E
:101E0000DBCF07F000500401856F0150866F025050
:101E1000876F0350886F045004018A6F05508B6FE1
:101E200006508C6F07508D6F0401855104018C039F
:101E3000F4CF01F0F3CF00F000500401906F015097
:101E4000916F0401855104018A03F4CF01F0F3CFAF
:101E500000F0005004018E6F01508F6F0401885113
:101E600004018A03F3CF00F00401915100260050D1
:101E7000916F0401875104018B03F3CF00F004013B
:101E8000915100260050916F0401875104018A038B
:101E9000F4CF01F0F3CF00F00401905100269151EE
:101EA00001220050906F0150916F0401865104018E
:101EB0008B03F4CF01F0F3CF00F004019051002622
:101EC000915101220050906F0150916F0401865191
:101ED00004018C03F3CF00F000500401F66F0401FD
:101EE000865104018A03F4CF01F0F3CF00F00050D3
:101EF0000401F46F0150F56F0401855104018D0355
:101F0000F3CF00F000500401FA6F04018551040181
:101F10008B03F4CF01F0F3CF00F000500401F86F11
:101F20000150F96F0401F36B0401F76B0401F351E5
:101F300004018E25006E0401F45104018F21016E0D
:101F40000401F55104019021026E0401F6510401CF
:101F50009121036E00508E6F01508F6F0250906F71
:101F60000350916F0401F75104018E25006E0401A6
:101F7000F85104018F21016E0401F95104019021EF
:101F8000026E0401FA5104019121036E03C0E9FFBE
:101F900002C0F4FF01C0F3FF0050E4CF07F0E4CF2C
:101FA00006F0E4CF05F0E4CF04F0E4CF03F0E4CF93
:101FB00002F0E4CF01F0E4CF00F0E4CFD9FF12004B
:101FC00000C0E5FF01C0E5FF02C0E5FF03C0E5FF7B
:101FD00004C0E5FF42EC22F0A8EC1EF0F3CF01F0C4
:101FE000F4CF02F0E9CF03F0880F0401346F130E31
:101FF0000120356F000E0220366F000E0320376F70
:1020000089EC16F09486820E006E0F0E016E0F0E94
:10201000036E380E0026035001220F0E036E800E51
:10202000005E0350015A820E026E0F0E036E0F0EF9
:10203000046E380E0226045003220F0E046E800E2A
:10204000025E0450035A02C0E9FF03C0EAFFEFCF6B
:1020500002F0028600C0E9FF01C0EAFF02C0EFFF04
:102060000F0EE56E000EE56A7BEC19F0E652E652C3
:102070009488820E006E0F0E016E0F0E036E380EE6
:102080000026035001220F0E036E800E005E0350E7
:10209000015A820E026E0F0E036E0F0E046E380E82
:1020A0000226045003220F0E046E800E025E0450BE
:1020B000035A02C0E9FF03C0EAFFEFCF02F0028833
:1020C00000C0E9FF01C0EAFF02C0EFFF100EE56E9D
:1020D000010EE56E7BEC19F0E652E652948A820E10
:1020E000006E0F0E016E0F0E036E380E00260350A9
:1020F00001220F0E036E800E005E0350015A820E05
:10210000026E0F0E036E0F0E046E380E0226045080
:1021100003220F0E046E800E025E0450035A02C0AA
:10212000E9FF03C0EAFFEFCF02F0028A00C0E9FF37
:1021300001C0EAFF02C0EFFF110EE56E020EE56E70
:102140007BEC19F0E652E652948C820E006E0F0E74
:10215000016E0F0E036E380E0026035001220F0E83
:10216000036E800E005E0350015A820E026E0F0E47
:10217000036E0F0E046E380E0226045003220F0E5B
:10218000046E800E025E0450035A02C0E9FF03C0D1
:10219000EAFFEFCF02F0028C00C0E9FF01C0EAFFC6
:1021A00002C0EFFF120EE56E030EE56E7BEC19F038
:1021B000E652E652E4CF04F0E4CF03F0E4CF02F0BD
:1021C000E4CF01F0E4CF00F01200430025630000EB
:1021D00000C0E5FF01C0E5FF0A014551D8B4F5D0C4
:1021E000A3A81DD0A4A81BD00A0160510A015D1943
:1021F00005E1CFEC21F00A015D6BE7D0000E0A018A
:102200006025006E016A0F0E012200C0E9FF01C0C7
:10221000EAFFEFCF33FF602B33CF73FFD6D0A4AAF2
:10222000D4D071A205D00A015E81CFEC21F0CDD0CF
:1022300071A405D00A015E83CFEC21F0C6D071A055
:102240003ED074CF33FF800E0A0146110F013319BF
:1022500004E10A015E897196B8D00F01335104E0A0
:1022600033510A01461927E10A015E9971960F015F
:10227000335103E00A015E9702D00A015E8733CF33
:1022800062FA35CF63FA0F0135050A01646F600EFB
:102290000A016325006E016A000E012200C0E9FFF9
:1022A00001C0EAFF33CFEFFF632B6351800A02E1E5
:1022B0000A01636B8AD00A015E99718686D074CF59
:1022C00033FF0A015EA919D0800E0A0146110F01E1
:1022D000331911E1899AA39A71980A015D5104E1B9
:1022E000736ACFEC21F007D000CF73FF010E0A0113
:1022F000606FA3886AD0718668D00F0133510A01DC
:1023000062270A0163510A0164191BE10A01625143
:102310000CE163CA35FF0A015EB712D0899AA39A0D
:102320007198736ACFEC21F00BD00A015E855EB71D
:1023300007D0899AA39A7198010E736ECFEC21F0A1
:1023400044D00A0163510F01361908E10F013651DB
:102350000F01351903E0CFEC21F037D035CF00F075
:10236000016A004A012AE56A800EE56E0150E56EB9
:102370000050E56E7AEC17F0006E040EE126005076
:102380000F01346F0A0163190CE11F0E0F013315A1
:102390000A01646F642B642B0F0135510A01642715
:1023A000649F63CA00F00A01632B016A600E002675
:1023B000000E012200C0E9FF01C0EAFF33CFEFFFAA
:1023C0006351800A02E10A01636BE4CF01F0E4CFBC
:1023D00000F01200D9CFE5FFE1CFD9FF00C0E5FF43
:1023E00001C0E5FF02C0E5FF03C0E5FF04C0E5FF53
:1023F00005C0E5FF06C0E5FF07C0E5FF08C0E5FF33
:1024000009C0E5FF0AC0E5FF0BC0E5FF0CC0E5FF12
:102410000DC0E5FF0EC0E5FF0FC0E5FF020EDBCFEC
:1024200000F0030EDBCF01F0040EDBCF02F0050E4F
:10243000DBCF03F0060EDBCF04F0070EDBCF05F099
:10244000080EDBCF06F0200E076E086A06C009F002
:102450000A6A0B6A0C6AE56AE56AE56A0950E56E84
:102460000350E56E0250E56E0150E56E0050E56EDA
:10247000C6EC12F00D6E080EE126300E0D263A0E57
:102480000D5C05E30D500E6E270E0E240D6EFF0E33
:1024900007260822200E07240E6E0A0E08200F6E53
:1024A0000EC0E9FF0FC0EAFF0DC0EFFF0C50E56E54
:1024B0000B50E56E0A50E56E0950E56E0350E56E6F
:1024C0000250E56E0150E56E0050E56EE6EC13F04B
:1024D000006EF3CF01F0F4CF02F0E9CF03F0080E65
:1024E000E1260050011002100310D8A4AFD707C096
:1024F00000F008C001F004C002F005C003F000C005
:1025000004F001C005F0004A012A200E04260A0E3C
:10251000052204C0E9FF05C0EAFFEFCF04F002C0C6
:10252000E9FF03C0EAFF04C0EFFF024A032A000EDE
:10253000015C02E1200E005CE2E302C0E9FF03C09F
:10254000EAFF000EEF6AE4CF0FF0E4CF0EF0E4CF25
:102550000DF0E4CF0CF0E4CF0BF0E4CF0AF0E4CFC1
:1025600009F0E4CF08F0E4CF07F0E4CF06F0E4CFC1
:1025700005F0E4CF04F0E4CF03F0E4CF02F0E4CFC1
:1025800001F0E4CF00F0E4CFD9FF1200D9CFE5FF8E
:10259000E1CFD9FF00C0E5FF01C0E5FF02C0E5FFC4
:1025A00003C0E5FF04C0E5FF05C0E5FF06C0E5FF89
:1025B00007C0E5FF08C0E5FF09C0E5FF0AC0E5FF69
:1025C000020EDBCF00F0030EDBCF01F0040EDBCFF9
:1025D00002F0050EDBCF03F0060EDBCF04F0070E92
:1025E000DBCF05F0080EDBCF06F0090EDBCF07F0DE
:1025F000086A096A0750800BE8440A6E0A501BE11A
:10260000045004260536063607360750035C08E1F9
:102610000650025C05E10550015C02E10450005CDB
:1026200006E2D890073206320532043204D0092A75
:1026300009C008F0DFD70750035C08E10650025CD0
:1026400005E10550015C02E10450005C08E3045020
:10265000005E0550015A0650025A0750035AD8909E
:10266000073206320532043208C009F00806095064
:10267000E2E103C0E9FF02C0F4FF01C0F3FF005034
:10268000E4CF0AF0E4CF09F0E4CF08F0E4CF07F09C
:10269000E4CF06F0E4CF05F0E4CF04F0E4CF03F09C
:1026A000E4CF02F0E4CF01F0E4CF00F0E4CFD9FFB3
:1026B000120000C0E5FF01C0E5FF03C0E5FF04C054
:1026C000E5FF05C0E5FF06C0E5FF07C0E5FF08C060
:1026D000E5FF09C0E5FF0AC0E5FF0BC0E5FF2CCF11
:1026E00000F02DCF01F00F012C3F01D02D2B005019
:1026F000E56EC1EC21F0E652076E046A056A066ACF
:102700002CCF00F02DCF01F00F012C3F01D02D2B4D
:102710000050E56EC1EC21F0E6520B6A0A6E086AC1
:102720000850041205120A5006120B5007122CCF43
:1027300000F02DCF01F00F012C3F01D02D2B0050C8
:10274000E56EC1EC21F0E652036E006A03C001F0B1
:10275000E86A03BEFF0E086E096E005004120150B5
:10276000051208500612095007122CCF00F02DCF89
:1027700001F00F012C3F01D02D2B0050E56EC1EC74
:1027800021F0E652016A04120150051206120712E6
:1027900007C0E9FF06C0F4FF05C0F3FF0450E4CF13
:1027A0000BF0E4CF0AF0E4CF09F0E4CF08F0E4CF77
:1027B00007F0E4CF06F0E4CF05F0E4CF04F0E4CF77
:1027C00003F0E4CF01F0E4CF00F01200D9CFE5FF31
:1027D000E1CFD9FF00C0E5FF01C0E5FF02C0E5FF82
:1027E00003C0E5FF04C0E5FF05C0E5FF06C0E5FF47
:1027F00007C0E5FF08C0E5FF09C0E5FF0AC0E5FF27
:102800000BC0E5FF0CC0E5FF0DC0E5FF020EDBCFFE
:1028100000F0030EDBCF01F0040EDBCF02F0050E5B
:10282000DBCF03F0060EDBCF04F0070EDBCF05F0A5
:10283000080EDBCF06F0090EDBCF07F0086A096A45
:102840000A6A0B6A200E0C6E0350800BE8440D6E72
:102850000050002601360236033608500826093695
:102860000A360B360D50D8A4088007500B5C08E1DF
:1028700006500A5C05E10550095C02E10450085C61
:1028800009E30450085E0550095A06500A5A0750D9
:102890000B5A00800C2ED8D703C0E9FF02C0F4FF0A
:1028A00001C0F3FF0050E4CF0DF0E4CF0CF0E4CF13
:1028B0000BF0E4CF0AF0E4CF09F0E4CF08F0E4CF66
:1028C00007F0E4CF06F0E4CF05F0E4CF04F0E4CF66
:1028D00003F0E4CF02F0E4CF01F0E4CF00F0E4CF66
:1028E000D9FF120000C0E5FF01C0E5FF02C0E5FF0F
:1028F00003C0E5FF04C0E5FF0F0136510F01351994
:1029000001E15CD036CF00F0002A009E600E00246A
:10291000016E026A000E022201C0E9FF02C0EAFF56
:10292000EFCF66FA1F0E0A01661736CF65FA6651B9
:102930000A016527652B652B659FD2EC1EF0016EA1
:10294000015003E1016A012A01D0016AD2EC1EF0B4
:102950000A01666F800E6615026E1F0E6615036E05
:1029600003C004F003C066FA045003E135CF36FF1C
:1029700038D001501BE002501FE0D2EC1EF0006E78
:102980000A0166070050420A17E000504E0A03E1B0
:1029900057EC1BF011D00050460A03E103EC22F083
:1029A0000BD00050490A08E1FF0006D036CF67FA85
:1029B0000250D8A446EC1DF065CA36FF0A01425108
:1029C0000A01431906E00A015D5103E1FCEC14F031
:1029D00008D089BA06D00A015D5103E172B2CFEC8A
:1029E00021F0E4CF04F0E4CF03F0E4CF02F0E4CF31
:1029F00001F0E4CF00F0120000C0E5FF01C0E5FFE8
:102A000002C0E5FF03C0E5FF72A276D003EC20F020
:102A1000006E005005E10A01436B0A01426B6CD065
:102A200043CA01F00050012603EC20F0026E0006BC
:102A30000250230A1FE1010E005CD8A05BD003EC1A
:102A400020F0026E690A03E14DEC1EF053D00250F3
:102A5000720A03E1CFEC21F04DD00250730A01E07D
:102A600049D0898A7186A38AA3987450745071984A
:102A7000718840D00250430A05E00250420A01E04A
:102A800039D001D0008E00C05FFA00500F01006FF6
:102A9000010E0A01606F0A014351011814E003ECB2
:102AA00020F0026E0A015F27000E0A016025006E09
:102AB000036A0F0E032200C0E9FF03C0EAFF02C051
:102AC000EFFF602BE8D7000E0A016025006E026A56
:102AD0000F0E02220A015F1D036E032A00C0E9FFE8
:102AE00002C0EAFF03C0EFFF0A01602B60CA5DFA73
:102AF0000F01316B01C043FAE4CF03F0E4CF02F0E1
:102B0000E4CF01F0E4CF00F01200D9CFE5FFE1CF30
:102B1000D9FF00C0E5FF01C0E5FF02C0E5FF03C02B
:102B2000E5FF04C0E5FF05C0E5FF06C0E5FF07C0FF
:102B3000E5FF020EDBCF00F0030EDBCF01F0040E49
:102B4000DBCF02F0050EDBCF03F002C006F006502B
:102B5000046E800A33E100C0E9FF01C0F3FF0250B8
:102B60005DEC20F0056EF3CF06F0F4CF07F003C064
:102B7000E5FF05C0E9FF06C0F3FF07500EEC22F0A9
:102B800000C0E9FF01C0F3FF02505DEC20F0056ECC
:102B9000F3CF06F0F4CF07F0052A02E3064A072A2E
:102BA00005C0E5FF06C0F4FF07C0F6FF00C0E9FF5F
:102BB00001C0F3FF0250B2EC21F01DD004AA1BD0DB
:102BC000047A045004E1035047EC22F014D004507E
:102BD000010A04E1035002EC00F00DD004500F0A8A
:102BE00004E103501CEC1EF006D004500E0A03E171
:102BF000035057EC22F0E4CF07F0E4CF06F0E4CF27
:102C000005F0E4CF04F0E4CF03F0E4CF02F0E4CF2A
:102C100001F0E4CF00F0E4CFD9FF1200D9CFE5FFF7
:102C2000E1CFD9FF00C0E5FF01C0E5FF02C0E5FF2D
:102C300003C0E5FF04C0E5FF05C0E5FF06C0E5FFF2
:102C400007C0E5FF020EDBCF00F0030EDBCF01F083
:102C5000040EDBCF02F0050EDBCF03F043CA44FACB
:102C60000A0142510A01445F440703C004F0056AA7
:102C7000030E0426D8B0052A44CA06F0076A075096
:102C8000800FF36E0550800FF35C02E10450065C88
:102C900002E2E8682BD0020E035C02E2E86A26D06A
:102CA00003060350E56E95EC1CF0E652046A0350EF
:102CB000045C14E204500024056EE86A0120066EEC
:102CC000E86A022005C0E9FF06C0F3FF81EC21F0AD
:102CD000042AE56E95EC1CF0E652E9D743CA44FAA3
:102CE0000A0142510A01445F4407E86AE4CF07F051
:102CF000E4CF06F0E4CF05F0E4CF04F0E4CF03F036
:102D0000E4CF02F0E4CF01F0E4CF00F0E4CFD9FF4C
:102D1000120000C0E5FF01C0E5FF02C0E5FF03C0EF
:102D2000E5FF04C0E5FF006A2E0E0024016E026A72
:102D30000F0E022201C0E9FF02C0EAFFEF6A002A7B
:102D4000020E005CF1E3006A016A026AE00E0124EF
:102D5000036E000E0220046E03C0E9FF04C0EAFF08
:102D6000EE6AEF6A5C0E0124036E040E0220046E0C
:102D700003C0E9FF04C0EAFFEE6AEF6A930E012484
:102D8000036E040E0220046E03C0E9FF04C0EAFFD4
:102D9000EE6AEF6AB30E0124036E040E0220046E85
:102DA00003C0E9FF04C0EAFFEE6AEF6AD30E012414
:102DB000036E040E0220046E03C0E9FF04C0EAFFA4
:102DC000EE687F0EEF6E020E0126D8B0022A002AAE
:102DD000100E005CD8A0BAD7AF0EC06EC16A010E4B
:102DE000C26EC282E4CF04F0E4CF03F0E4CF02F07D
:102DF000E4CF01F0E4CF00F012004320412025642D
:102E00002025640A0000D9CFE5FFE1CFD9FF00C03B
:102E1000E5FF01C0E5FF02C0E5FF03C0E5FF04C018
:102E2000E5FF05C0E5FF020EDBCF00F0030EDBCFB0
:102E300001F0040EDBCF02F00050020DF450036EDF
:102E4000F3CF00F05C0E0024046E040E0320056E28
:102E500004C0E9FF05C0EAFF01C0EEFF02C0EFFFBA
:102E6000930E0024046E040E0320056E04C0E9FFD7
:102E700005C0EAFFEECF04F0EFCF05F00150045C8F
:102E8000016E02500558026E000E00260A0E032243
:102E900000C0E9FF03C0EAFF01C0EEFF02C0EFFF80
:102EA000D88002AED89004E3021E016CD8B4022A86
:102EB0000250800F800F02E1030E015C02E2016A02
:102EC000026A0150021007E100C0E9FF03C0EAFFF7
:102ED000000EEE6AEF6AE4CF05F0E4CF04F0E4CF31
:102EE00003F0E4CF02F0E4CF01F0E4CF00F0E4CF50
:102EF000D9FF1200D9CFE5FFE1CFD9FF00C0E5FF30
:102F000001C0E5FF02C0E5FF03C0E5FF04C0E5FF27
:102F100005C0E5FF06C0E5FF020EDBCF00F0030EA3
:102F2000DBCF01F0040EDBCF02F0050EDBCF03F0A8
:102F3000D88001AED890046A0436045007E0011C22
:102F4000066E001C056E054A062A04D000C005F076
:102F500001C006F0D88003AED89007E3031C016ED1
:102F6000021C006E004A012A04D002C000F003C017
:102F700001F00150E56E0050E56E0650E56E05501B
:102F8000E56E1EEC19F0006EF3CF01F0040EE126A1
:102F900004500AE0011C036E001C026E024A032A60
:102FA00003C0F3FF025003D001C0F3FF0050E4CF91
:102FB00006F0E4CF05F0E4CF04F0E4CF03F0E4CF73
:102FC00002F0E4CF01F0E4CF00F0E4CFD9FF12002B
:102FD000D9CFE5FFE1CFD9FF00C0E5FF01C0E5FF94
:102FE00002C0E5FF03C0E5FF04C0E5FF05C0E5FF43
:102FF000020EDBCF00F0030EDBCF01F0040EDBCFBF
:1030000002F0050EDBCF03F02CCF04F02DCF05F03E
:103010000F012C3F01D02D2B0350E56E0450E56EBF
:1030200023EC1FF0E652E6522CCF04F02DCF05F032
:103030000F012C3F01D02D2B0250056EE56E045080
:10304000E56E23EC1FF0E652E6522CCF04F02DCFB4
:1030500005F00F012C3F01D02D2B0150056EE56EC0
:103060000450E56E23EC1FF0E652E6522CCF04F03C
:103070002DCF05F00F012C3F01D02D2B0050E56E18
:103080000450E56E23EC1FF0E652E652E4CF05F063
:10309000E4CF04F0E4CF03F0E4CF02F0E4CF01F09A
:1030A000E4CF00F0E4CFD9FF1200D9CFE5FFE1CFA4
:1030B000D9FF00C0E5FF01C0E5FF02C0E5FF03C086
:1030C000E5FF04C0E5FF05C0E5FF06C0E5FF020E11
:1030D000DBCF00F0030EDBCF01F0040EDBCF02F0FC
:1030E0000F01305119E159EC13F0036EF3CF04F0E6
:1030F000F4CF05F0E9CF06F003C0E5FF04C0F4FF0C
:1031000005C0F6FF06C0F7FF00C0E9FF01C0F3FFEE
:10311000025092EC21F01ED00F013051010A1AE149
:1031200000C0E9FF01C0F3FF0250E3EC1FF0006EA6
:10313000F3CF01F0F4CF02F0E9CF03F00350E56ED6
:103140000250E56E0150E56E0050E56EE8EC17F0B8
:10315000040EE126E4CF06F0E4CF05F0E4CF04F05E
:10316000E4CF03F0E4CF02F0E4CF01F0E4CF00F0CD
:10317000E4CFD9FF1200D9CFE5FFE1CFD9FF00C0DE
:10318000E5FF01C0E5FF02C0E5FF03C0E5FF04C0A5
:10319000E5FF05C0E5FF06C0E5FF020EDBCF00F04E
:1031A000030EDBCF01F0040EDBCF02F0050EDBCF08
:1031B00003F0060EDBCF04F0070EDBCF05F0080EA0
:1031C000DBCF06F0D88003AED89015E306500A0A8C
:1031D00012E104C0E9FF05C0EAFF2D0EEF6E044ABC
:1031E000052A031E021E011E006C05E1012A03E1EF
:1031F000022AD8B4032A0650E56E0550E56E045045
:10320000E56E0350E56E0250E56E0150E56E00502C
:10321000E56EEAEC11F0070EE126E4CF06F0E4CF0C
:1032200005F0E4CF04F0E4CF03F0E4CF02F0E4CF04
:1032300001F0E4CF00F0E4CFD9FF1200D9CFE5FFD1
:10324000E1CFD9FF00C0E5FF01C0E5FF02C0E5FF07
:1032500003C0E5FF04C0E5FF05C0E5FF06C0E5FFCC
:10326000020EDBCF00F0030EDBCF01F0040EDBCF4C
:1032700002F0050EDBCF03F0046A056A0350800BF1
:10328000E844066E065011E1025002260336035050
:10329000015C02E10250005C04E2D8900332023289
:1032A00004D0052A05C004F0E9D70350015C02E10F
:1032B0000250005C04E30250005E0350015AD890B3
:1032C0000332023204C005F004060550EEE101C0ED
:1032D000F3FF0050E4CF06F0E4CF05F0E4CF04F0B4
:1032E000E4CF03F0E4CF02F0E4CF01F0E4CF00F04C
:1032F000E4CFD9FF1200D9CFE5FFE1CFD9FF00C05D
:10330000E5FF01C0E5FF02C0E5FF03C0E5FF04C023
:10331000E5FF05C0E5FF06C0E5FF020EDBCF00F0CC
:10332000030EDBCF01F00038E8441F0B026E036A86
:103330002E0E02260F0E032202C0E9FF03C0EAFF91
:10334000EFCF04F0070E0014056E010E066E055057
:1033500005E0E86CD8900636010FFDE30650041234
:1033600002C0E9FF03C0EAFF04C0EFFF026A240EB7
:103370000026040E022200C0E9FF02C0EAFF01C0DD
:10338000EFFFE4CF06F0E4CF05F0E4CF04F0E4CFA4
:1033900003F0E4CF02F0E4CF01F0E4CF00F0E4CF9B
:1033A000D9FF120000C0E5FF01C0E5FF02C0E5FF44
:1033B00003C0E5FF36CF00F0016A67CA02F0036A76
:1033C0000250005E0350015AE56A800EE56E01501E
:1033D000E56E0050E56E7AEC17F0006E040EE12603
:1033E000000667CA01F0430E1CEC1EF0200E1CEC18
:1033F0001EF00050800F7F0F20E3600E0124026E4C
:10340000036A000E032202C0E9FF03C0EAFFEFCF08
:1034100002F0E56A0250E56E000EE56E430EE56EC1
:10342000B60EE56ED9EC1BF0050EE126012A01501F
:10343000800A01E1016A0006DCD7E4CF03F0E4CFA3
:1034400002F0E4CF01F0E4CF00F01200D9CFE5FFA5
:10345000E1CFD9FF00C0E5FF01C0E5FF02C0E5FFF5
:1034600003C0E5FF04C0E5FF020EDBCF00F0030E52
:10347000DBCF01F0040EDBCF02F00F01305111E180
:10348000B6EC1DF0036EF3CF04F003C0E5FF04C0FB
:10349000F4FF00C0E9FF01C0F3FF0250EBEC21F0A4
:1034A00016D00F013051010A12E100C0E9FF01C03E
:1034B000F3FF02501CEC21F0006EF3CF01F001503D
:1034C000E56E0050E56E58EC1CF0E652E652E4CF93
:1034D00004F0E4CF03F0E4CF02F0E4CF01F0E4CF56
:1034E00000F0E4CFD9FF1200760EF66E440EF76EB0
:1034F000000EF86E0900F550056E0900F550066ED5
:1035000004E1056702D0C1EF1AF00900F550006E22
:103510000900F550016E0900F550026E090009001E
:10352000F550E96E0900F550EA6E0900090009003E
:10353000F550036E0900F550046E09000900F6CF3E
:1035400007F0F7CF08F0F8CF09F000C0F6FF01C090
:10355000F7FF02C0F8FF035002E1045007E0090042
:10356000F550EE6E0306F8E20406F9D707C0F6FF41
:1035700008C0F7FF09C0F8FF050601E2060680EF64
:103580001AF01200D9CFE5FFE1CFD9FF00C0E5FF67
:1035900001C0E5FF02C0E5FF03C0E5FF04C0E5FF91
:1035A00005C0E5FF020EDBCF00F00050010A24E168
:1035B000016A026A036AB30E0224046E040E032039
:1035C000056E04C0E9FF05C0EAFFEE687F0EEF6EEE
:1035D000D30E0224046E040E0320056E04C0E9FF1E
:1035E00005C0EAFFEE6AEF6A020E0226D8B0032A8F
:1035F000012A100E015CDFE300C048FAE4CF05F0B9
:10360000E4CF04F0E4CF03F0E4CF02F0E4CF01F024
:10361000E4CF00F0E4CFD9FF120000C0E5FF01C005
:10362000E5FF02C0E5FF03C0E5FF72EC14F097EC84
:103630000CF0A8EC1EF0006EF3CF01F0F4CF02F016
:10364000E9CF03F004013451005E3551015A36517F
:10365000025A3751035A039E3F0E035C08E1FF0EE6
:10366000025C05E1FF0E015C02E1FF0E005C16E268
:10367000A8EC1EF0F3CF01F0F4CF02F0E9CF03F095
:10368000880F0401346F130E0120356F000E0220E5
:10369000366F000E0320376FC1EC07F0E4CF03F064
:1036A000E4CF02F0E4CF01F0E4CF00F0120000C05C
:1036B000E5FF01C0E5FF02C0E5FFD2EC1EF0006EA1
:1036C000D2EC1EF0016E0050026ED00E0224006E8D
:1036D0000A0E005C05E30050026EF90E0224006E33
:1036E0000150026ED00E0224016E0A0E015C05E349
:1036F0000150026EF90E0224016E080E005C12E207
:10370000100E015CD8B00ED00038F00B0124006E12
:103710000CEC1DF0016E015005E10050E56E92ECDD
:1037200020F0E652E4CF02F0E4CF01F0E4CF00F065
:103730001200D9CFE5FFE1CFD9FF00C0E5FF01C0FE
:10374000E5FF02C0E5FF03C0E5FF04C0E5FF020E90
:10375000DBCF00F00038E8441F0B016E026A2E0E2A
:1037600001260F0E022201C0E9FF02C0EAFFEFCFDF
:1037700003F0070E0016010E046E005005E0E86C21
:10378000D8900436010FFDE3041C031601C0E9FFC5
:1037900002C0EAFF03C0EFFFE4CF04F0E4CF03F080
:1037A000E4CF02F0E4CF01F0E4CF00F0E4CFD9FFA2
:1037B0001200D9CFE5FFE1CFD9FF00C0E5FF01C07E
:1037C000E5FF02C0E5FF020ED924006E000EDA20EC
:1037D000016E800E026E030E0026000E01220222F0
:1037E0000250E56E0150E56E0050E56E040EDBCF31
:1037F000E5FF030EDBCFE5FF020EDBCFE5FF0F0198
:103800002551E56E2451E56E2351E56E0EEC00F076
:10381000006EF3CF01F0090EE12601C0F3FF005066
:10382000E4CF02F0E4CF01F0E4CF00F0E4CFD9FF21
:103830001200D9CFE5FFE1CFD9FF00C0E5FF01C0FD
:10384000E5FF02C0E5FF03C0E5FF020EDBCF00F09D
:10385000030EDBCF01F0040EDBCF02F00F0130517D
:103860000DE1F0EC20F0036E03C0E5FF00C0E9FFBE
:1038700001C0F3FF02500EEC22F00FD00F013051C7
:10388000010A0BE100C0E9FF01C0F3FF025081EC27
:1038900021F0E56E98EC1FF0E652E4CF03F0E4CFA0
:1038A00002F0E4CF01F0E4CF00F0E4CFD9FF120042
:1038B000D9CFE5FFE1CFD9FF00C0E5FF01C0E5FFAB
:1038C00002C0E5FF03C0E5FF020EDBCF00F0030EF0
:1038D000DBCF01F02CCF02F02DCF03F00F012C3FF6
:1038E00001D02D2B0150E56E0250E56E23EC1FF048
:1038F000E652E6522CCF02F02DCF03F00F012C3F01
:1039000001D02D2B0050E56E0250E56E23EC1FF028
:10391000E652E652E4CF03F0E4CF02F0E4CF01F048
:10392000E4CF00F0E4CFD9FF1200D9CFE5FFE1CF1B
:10393000D9FF00C0E5FF01C0E5FF02C0E5FF03C0FD
:10394000E5FF04C0E5FF020EDBCF00F042CA01F044
:10395000026A014A022A43CA03F0046A01500318AA
:1039600003E10250041801E001D00ED0000E0A015C
:103970004225016E026A070E022201C0E9FF02C061
:10398000EAFF00C0EFFF422BE4CF04F0E4CF03F0E6
:10399000E4CF02F0E4CF01F0E4CF00F0E4CFD9FFB0
:1039A0001200D9CFE5FFE1CFD9FF00C0E5FF01C08C
:1039B000E5FF02C0E5FF03C0E5FF020EDBCF00F02C
:1039C000016A67CA02F0036A02500026035001220E
:1039D000E56A800EE56E0150E56E0050E56E7AEC0A
:1039E00017F0006EF3CF01F0040EE126600E002602
:1039F000000E012200C0E9FF01C0EAFFEFCF00F096
:103A00000050E4CF03F0E4CF02F0E4CF01F0E4CFC4
:103A100000F0E4CFD9FF120000C0E5FF01C0E5FFD0
:103A200002C0E5FF010E006ED2EC1EF0016E01C077
:103A300002F0015023E00050E56EC1EC21F0016E70
:103A4000E652015010E10A0E005C0BE20A0E006E15
:103A5000E56EC1EC21F0016EE652015004E1E86828
:103A60000ED0E8680CD00150021802E0E86807D0D8
:103A7000002A1B0E005CD8E3E86801D0E86AE4CFB6
:103A800002F0E4CF01F0E4CF00F0120000C0E5FF47
:103A900001C0E5FFD2EC1EF0006E4C0A03E1D2EC4F
:103AA0001EF027D00050450A24E1000EE56E210EDD
:103AB000E56ECA0EE56ED9EC1BF0030EE12651EC63
:103AC00022F0006E00C001F0000601500FE0D2ECC1
:103AD0001EF0E56AE56E000EE56E210EE56ECC0E79
:103AE000E56ED9EC1BF0050EE126ECD70A0E1CECB6
:103AF0001EF0E4CF01F0E4CF00F01200F3CFE5FFB9
:103B0000F4CFE5FFE9CFE5FFEACFE5FFFACFE5FF28
:103B1000FBCFE5FF0A01405104017E6F0A014151CC
:103B200004017F6FD6507C6FD7507D6FF2A411D007
:103B30000A01403F01D0412BF2940A014051040197
:103B40007E6F0A01415104017F6FD6507C6FD750C0
:103B50007D6FE4CFFBFFE4CFFAFFE4CFEAFFE4CFD1
:103B6000E9FFE4CFF4FFE4CFF3FF110000C0E5FF6D
:103B700001C0E5FF02C0E5FF03C0E5FF2CCF00F068
:103B80002DCF01F00F012C3F01D02D2B0050E56E01
:103B9000C1EC21F0E652036E026A2CCF00F02DCF6B
:103BA00001F00F012C3F01D02D2B0050E56EC1EC30
:103BB00021F0E652016A02120150031203C0F3FF22
:103BC0000250E4CF03F0E4CF02F0E4CF01F0E4CF01
:103BD00000F01200D9CFE5FFE1CFD9FF00C0E5FF2B
:103BE00001C0E5FF02C0E5FF03C0E5FF04C0E5FF3B
:103BF000020EDBCF00F0030EDBCF01F0040EDBCFB3
:103C000002F0050EDBCF03F0060EDBCFE9FF070E57
:103C1000DBCFEAFF080EDBCF04F040EC04F0E4CF8A
:103C200004F0E4CF03F0E4CF02F0E4CF01F0E4CFFE
:103C300000F0E4CFD9FF120000C0E5FF01C0E5FFAE
:103C400002C0E5FF006E390E0A014725016E026AC7
:103C5000040E022201C0E9FF02C0EAFF00C0EFFF2C
:103C6000220E475D01E2472B00500A0A0FE10A01CC
:103C70004751E56E800EE56E040EE56E390EE56E79
:103C80000EEC16F0040EE1260A01476BE4CF02F0B9
:103C9000E4CF01F0E4CF00F012000A01426B0A0108
:103CA000436B0A014469898A929A766A3F0E756E5F
:103CB0007086728A7284728C7290718C718E0A0115
:103CC0005E6B0F01326B0F01356B0F01366B0A0112
:103CD0005D6B000EE56AC1EC21F00A01466FE65209
:103CE000A598A59A010E0A01456F0F01236B246B5D
:103CF0002F0E256FCFEC21F01200D9CFE5FFE1CFD9
:103D0000D9FF00C0E5FF01C0E5FF02C0E5FF03C029
:103D1000E5FF020EDBCF00F0030EDBCF01F0040E57
:103D2000DBCF02F0050EDBCF03F0060EDBCFE9FFA1
:103D3000070EDBCFEAFF00EC0AF0E4CF03F0E4CF9C
:103D400002F0E4CF01F0E4CF00F0E4CFD9FF12009D
:103D50000A0140510401836F0A0141510401846F3B
:103D6000D650816FD750826F83510A01401905E107
:103D7000040184510A0141190CE00A014051040177
:103D8000836F0A0141510401846FD650816FD7506F
:103D9000826F84C4E9FF83C4F4FF82C4F3FF04018B
:103DA0008151120000C0E5FF01C0E5FF0F0136514F
:103DB0000A01651905E00F0136510F01351902E1BD
:103DC000E86A15D036CF00F00F01362B016A600E7D
:103DD0000026000E012200C0E9FF01C0EAFFEFCF7C
:103DE00000F03651800A02E10F01366B0050E4CF3B
:103DF00001F0E4CF00F0120000C0E5FF4BEC22F030
:103E00000401896B806B8983006A89B3002A0050A2
:103E1000010BE844F46E8051FD0BF410806FD58ED9
:103E2000D59CD59AD588D596D594D582D580F28A59
:103E3000F184D08EF28EF28CBA80FF0EBB68BA8409
:103E4000E4CF00F01200D9CFE5FFE1CFD9FF00C0E9
:103E5000E5FF020EDBCF00F0030EDBCFA8FF00C0B2
:103E6000A9FFA69EA69CA684F29EF29C550EA76E64
:103E7000AA0EA76EA682A6A202D00000FCD7E86A0E
:103E8000A6B6E82AA694F28EF28CE4CF00F0E4CF36
:103E9000D9FF1200D9CFE5FFE1CFD9FF00C0E5FF80
:103EA00001C0E5FF020EDBCF00F00050020DF45020
:103EB000016EF3CF00F0000E00260A0E012200C0B2
:103EC000E9FF01C0EAFFEECF00F0EFCF01F001C043
:103ED000F3FF0050E4CF01F0E4CF00F0E4CFD9FFCE
:103EE0001200D9CFE5FFE1CFD9FF00C0E5FF01C047
:103EF000E5FF020EDBCF00F00050020DF450016E22
:103F0000F3CF00F0E00E0026000E012200C0E9FF12
:103F100001C0EAFFEECF00F0EFCF01F001C0F3FFE8
:103F20000050E4CF01F0E4CF00F0E4CFD9FF12005D
:103F3000D9CFE5FFE1CFD9FF00C0E5FF01C0E5FF24
:103F400002C0E5FF020EDBCF00F02CCF01F02DCF39
:103F500002F00F012C3F01D02D2B0050E56E0150D7
:103F6000E56E23EC1FF0E652E652E4CF02F0E4CF18
:103F700001F0E4CF00F0E4CFD9FF1200D8CFE5FF85
:103F8000E0CFE5FFE56EF3CFE5FFF4CFE5FFE9CF46
:103F9000E5FFEACFE5FFFACFE5FFFBCFE5FFE8EC71
:103FA00010F0E4CFFBFFE4CFFAFFE4CFEAFFE4CF69
:103FB000E9FFE4CFF4FFE4CFF3FFE450E4CFE0FF08
:103FC000E4CFD8FF1000E8AE0AD0F3CFEAFFEE50FE
:103FD000EECFF3FFEECFF4FFEECFE9FF1200E8BC27
:103FE00064EF22F0E9CFF6FFF3CFF7FFF86E090098
:103FF000F5500900F5CFF3FF0900F5CFF4FF0900F4
:10400000F5CFE9FF120000C0E5FF01C0E5FF0A019E
:1040100042510A01431902E1E86A0FD0000E0A0179
:104020004325006E016A070E012200C0E9FF01C0AE
:10403000EAFFEFCF00F0432B0050E4CF01F0E4CFD4
:1040400000F01200F2CFEAFFF29EA69EA69CA68484
:10405000E9CFA9FFF3CFAAFFE4CFA8FF23EC22F01A
:10406000F4CFA8FF23EC22F0F6CFA8FF23EC22F038
:10407000F7CFA8FF23EC22F0A694EABEF28E12003E
:10408000F2CFF6FFF29EA69EA69CE9CFA9FFF3CF42
:10409000AAFFA680A850A94AAA2AA680A8CFF3FF03
:1040A000A94AAA2AA680A8CFF4FFA94AAA2AA680CC
:1040B000A8CFEAFFF6BEF28E1200E8AE08D0F3CF2A
:1040C000EAFFEE50EECFF3FFEECFF4FF1200E8BCB4
:1040D00066EF22F0E9CFF6FFF3CFF7FFF86E0900A5
:1040E000F5500900F5CFF3FF0900F5CFF4FF1200FA
:1040F000F2CFEAFFF29EA69EA69CA684E9CFA9FF76
:10410000F3CFAAFFE4CFA8FF23EC22F0F4CFA8FF5F
:1041100023EC22F0F6CFA8FF23EC22F0A694EABE0F
:10412000F28E1200D9CFE5FFE1CFD9FF00C0E5FF45
:10413000020EDBCF00F000C046FA0050E56E000E24
:10414000E56A23EC1FF0E652E652E4CF00F0E4CF3C
:10415000D9FF1200F2CFF6FFF29EA69EA69CE9CFF1
:10416000A9FFF3CFAAFFA680A850A94AAA2AA68031
:10417000A8CFF3FFA94AAA2AA680A8CFF4FFF6BECB
:10418000F28E120000C0E5FF01C0E5FF600E0F01D6
:104190003625006E016A000E012200C0E9FF01C051
:1041A000EAFFEFCF00F00050E4CF01F0E4CF00F0E1
:1041B0001200D9CFE5FFE1CFD9FF00C0E5FF020E25
:1041C000DBCF00F0610E005C05E37B0E005C02E2D9
:1041D000010E01D0E86AE4CF00F0E4CFD9FF12006D
:1041E00000C0E5FF01C0E5FF2CCF00F02DCF01F0AE
:1041F0000F012C3F01D02D2B0050E56EC1EC21F0BA
:10420000E652E4CF01F0E4CF00F01200D9CFE5FF91
:10421000E1CFD9FF00C0E5FF020EDBCF00F000C008
:1042200045FA005004E1CFEC21F0A39AA398E4CF23
:1042300000F0E4CFD9FF1200E8AE06D0F3CFEAFFDA
:10424000EE50EECFF3FF1200E8BC62EF22F0E9CFB0
:10425000F6FFF3CFF7FFF86E0900F5500900F5CF30
:10426000F3FF1200F2CFEAFFF29EA69EA69CA68460
:10427000E9CFA9FFF3CFAAFFE4CFA8FF23EC22F0F8
:10428000F4CFA8FF23EC22F0A694EABEF28E12002F
:1042900018EEFFF028EEFFF0F86AA68EA69CE968FB
:1042A0000E0EEA6E0068000EED6A0050FDE174EC3F
:1042B0001AF006EC00F0FFD7F2CFF6FFF29EA69EB2
:1042C000A69CE9CFA9FFF3CFAAFFA680A850A94AD0
:1042D000AA2AA680A8CFF3FFF6BEF28E1200F2CF74
:1042E000EAFFF29EA69EA69CA684E9CFA9FFF3CF83
:1042F000AAFFE4CFA8FF23EC22F0A694EABEF28E38
:104300001200E8AE04D0F3CFEAFFEE501200E8BC92
:1043100060EF22F0E9CFF6FFF3CFF7FFF86E090068
:10432000F5501200E8AE0BD0F3CFEAFFE4CFEEFF7A
:10433000F4CFEEFFF6CFEEFFF7CFEEFF1200E8BCB2
:104340005EEF22F0120000000000FF0000000002FB
:104350000002000000420000000000000000000019
:1043600000000000E8AE09D0F3CFEAFFE4CFEEFF93
:10437000F4CFEEFFF6CFEEFF1200E8BC68EF22F0BC
:104380001200D9CFE5FFE1CFD9FF020EDBCFA9FFA5
:10439000A69CA69EA680A850E4CFD9FF120072A2C8
:1043A000FED7898A745000007450719871887186A4
:1043B000A38AA398120025642000F2CFF6FFF29E94
:1043C000A69EA69CE9CFA9FFF3CFAAFFA680A8507E
:1043D000F6BEF28E1200E8AE07D0F3CFEAFFE4CFCC
:1043E000EEFFF4CFEEFF1200E8BC5CEF22F012000B
:1043F000700ED36E9B8CFF0E9268936894689668DB
:10440000626AF19E120000C0E5FF0CEC1DF0006E28
:10441000005001E1FF00E4CF00F01200E8AE05D04B
:10442000F3CFEAFFE4CFEEFF1200E8BC5AEF22F030
:104430001200D9CFE5FFE1CFD9FF020EDBCF4BFA57
:10444000E4CFD9FF1200550EA76EAA0EA76EA68262
:10445000A6B2FED7A94AAA2A010E0F01306F1C0E80
:104460000F012C6F2D6B12000F01306B1C0E0F0112
:104470002C6F2D6B1200010046430000400A000023
:104480001D000000FCEC1EF04DEC1EF01200ACA272
:10449000FED7AD6E1200F8EC21F012000F0136517C
:1044A00012000A01665112000A0145511200E8CFBC
:1044B0007FFF12006FEF21F032EF21F022EF20F0AA
:1044C000DDEF21F05CEF21F040EF20F0AAEF20F0CB
:0444D00078EF20F071
:00000001FF
